:020000040000FA
:040000000FEF0BF003
:04000800F0EF09F01C
:06002A00D9CFE5FFE1CF94
:10003000D9FF00C0E5FF01C0E5FF02C0E5FF03C036
:10004000E5FF04C0E5FF05C0E5FF06C0E5FF07C00A
:10005000E5FF08C0E5FF09C0E5FF0AC0E5FF020EA5
:10006000DBCF00F0030EDBCF01F0040EDBCF02F09C
:10007000050EDBCF03F0060EDBCF04F0070EDBCF5F
:1000800005F000C006F001C007F002C008F0035000
:1000900003E003500508036E270EE56E100EE56EB3
:1000A0000550E56E0450E56ED0EC05F0096EF3CF17
:1000B0000AF0040EE126300E092609C0E5FF06C04D
:1000C000E9FF07C0F3FF08501BEC0BF0062AD8B07D
:1000D000072AD8B0082A030603500EE12E0EE56E5B
:1000E00006C0E9FF07C0F3FF08501BEC0BF0062A1F
:1000F000D8B0072AD8B0082A270EE56E100EE56E94
:100100000550E56E0450E56E74EC05F0046EF3CF17
:1001100005F0040EE126030EE56EE80EE56E0550CF
:10012000E56E0450E56ED0EC05F0096EF3CF0AF0F1
:10013000040EE126300E092609C0E5FF06C0E9FFDE
:1001400007C0F3FF08501BEC0BF0062AD8B0072AB3
:10015000D8B0082A030603500EE12E0EE56E06C045
:10016000E9FF07C0F3FF08501BEC0BF0062AD8B0DC
:10017000072AD8B0082A030EE56EE80EE56E055092
:10018000E56E0450E56E74EC05F0046EF3CF05F0F7
:10019000040EE126000EE56E640EE56E0550E56E78
:1001A0000450E56ED0EC05F0096EF3CF0AF0040EB2
:1001B000E126300E092609C0E5FF06C0E9FF07C0A9
:1001C000F3FF08501BEC0BF0062AD8B0072AD8B072
:1001D000082A030603500EE12E0EE56E06C0E9FF65
:1001E00007C0F3FF08501BEC0BF0062AD8B0072A13
:1001F000D8B0082A000EE56E640EE56E0550E56E77
:100200000450E56E74EC05F0046EF3CF05F0040EB7
:10021000E126000EE56E0A0EE56E0550E56E04500F
:10022000E56ED0EC05F0096EF3CF0AF0040EE1267E
:10023000300E092609C0E5FF06C0E9FF07C0F3FF3D
:1002400008501BEC0BF0062AD8B0072AD8B0082AB1
:10025000030603500EE12E0EE56E06C0E9FF07C04F
:10026000F3FF08501BEC0BF0062AD8B0072AD8B0D1
:10027000082A000EE56E0A0EE56E0550E56E045084
:10028000E56E74EC05F0046EF3CF05F0040EE12684
:10029000300E042604C0E5FF06C0E9FF07C0F3FFE7
:1002A00008501BEC0BF0062AD8B0072AD8B0082A51
:1002B000032E09D02E0EE56E06C0E9FF07C0F3FF3E
:1002C00008501BEC0BF00050040F036E000E0120D1
:1002D000046E000E0220056E0250800FF36E055072
:1002E000800FF35C05E10450015C02E10350005C07
:1002F00019E200C0E9FF01C0F3FF0250C4EC0AF0AC
:10030000066E300A0FE1200EE56E00C0E9FF01C065
:10031000F3FF02501BEC0BF0002AD8B0012AD8B032
:10032000022ADAD7E4CF0AF0E4CF09F0E4CF08F0EC
:10033000E4CF07F0E4CF06F0E4CF05F0E4CF04F01B
:10034000E4CF03F0E4CF02F0E4CF01F0E4CF00F01B
:10035000E4CFD9FF1200D9CFE5FFE1CFD9FF00C02C
:10036000E5FF01C0E5FF02C0E5FF03C0E5FF04C0F3
:10037000E5FF05C0E5FF06C0E5FF07C0E5FF020E8B
:10038000DBCF00F0030EDBCF01F0040EDBCF02F079
:10039000050EDBCF03F0640EE56E03C0E5FFEDEC68
:1003A00008F0046EE450E450300E042604C0E5FF6B
:1003B00000C0E9FF01C0F3FF02501BEC0BF000503E
:1003C000010F046E000E0120056E000E0220066E65
:1003D000640EE56E03C0E5FF43EC08F0036EE450E5
:1003E000E4500A0EE56E03C0E5FFEDEC08F0076E81
:1003F000E450E450300E072607C0E5FF04C0E9FFD3
:1004000005C0F3FF06501BEC0BF0042AD8B0052AF8
:10041000D8B0062A0A0EE56E03C0E5FF43EC08F0EB
:10042000036EE450E450300E032603C0E5FF04C021
:10043000E9FF05C0F3FF06501BEC0BF00050020F64
:10044000036E000E0120046E000E0220056E0250A5
:10045000800FF36E0550800FF35C05E10450015CE2
:1004600002E10350005C19E200C0E9FF01C0F3FFA4
:100470000250C4EC0AF0066E300A0FE1200EE56E61
:1004800000C0E9FF01C0F3FF02501BEC0BF0002A93
:10049000D8B0012AD8B0022ADAD7E4CF07F0E4CFE7
:1004A00006F0E4CF05F0E4CF04F0E4CF03F0E4CFAE
:1004B00002F0E4CF01F0E4CF00F0E4CFD9FF120066
:1004C000D9CFE5FFE1CFD9FF00C0E5FF01C0E5FFCF
:1004D00002C0E5FF03C0E5FF04C0E5FF05C0E5FF7E
:1004E00006C0E5FF07C0E5FF08C0E5FF020EDBCF51
:1004F00000F0030EDBCF01F0040EDBCF02F0050E9F
:10050000DBCF03F0060EDBCF04F0070EDBCF05F0E8
:10051000080EDBCF06F0090EDBCF07F01AEC0AF06D
:1005200003A003D0020EC86E02D0090EC86E56ECAE
:100530000BF00050E56E03EC0BF0E12A03A208D0AB
:100540000250036E086A0350E56E03EC0BF0E12ADB
:100550000150E56E03EC0BF0E12A50EC0BF000804B
:100560000050E56E03EC0BF0E12A04C000F005C07A
:1005700001F006C002F007C003F0020E035C16E3B0
:10058000010EE56E69EC0AF0046EE12A04C0E5FF95
:1005900000C0E9FF01C0F3FF02501BEC0BF0002A82
:1005A000D8B0012AD8B0022A0306E7D703500FE0DB
:1005B000000EE56E69EC0AF0036EE12A03C0E5FF68
:1005C00000C0E9FF01C0F3FF02501BEC0BF04AEC46
:1005D0000BF0E86AE4CF08F0E4CF07F0E4CF06F0D0
:1005E000E4CF05F0E4CF04F0E4CF03F0E4CF02F071
:1005F000E4CF01F0E4CF00F0E4CFD9FF1200D9CF6F
:10060000E5FFE1CFD9FF00C0E5FF01C0E5FF02C073
:10061000E5FF03C0E5FF04C0E5FF05C0E5FF06C038
:10062000E5FF07C0E5FF08C0E5FF09C0E5FF0AC018
:10063000E5FF0BC0E5FF0CC0E5FF0DC0E5FF020EB6
:10064000DBCF00F0030EDBCF01F0040EDBCF02F0B6
:10065000050EDBCF03F0060EDBCF04F0070EDBCF79
:1006600005F0080EDBCF06F0090EDBCF07F0086AB5
:10067000096A0A6A0B6A200E0C6E0344010B0D6EA8
:10068000010E0D16005000260136023603360850C2
:10069000082609360A360B360D50D8A408800750B4
:1006A0000B5C08E106500A5C05E10550095C02E1BB
:1006B0000450085C09E30450085E0550095A0650CE
:1006C0000A5A07500B5A00800C2ED7D703C0E9FFF7
:1006D00002C0F4FF01C0F3FF0050E4CF0DF0E4CFFF
:1006E0000CF0E4CF0BF0E4CF0AF0E4CF09F0E4CF54
:1006F00008F0E4CF07F0E4CF06F0E4CF05F0E4CF54
:1007000004F0E4CF03F0E4CF02F0E4CF01F0E4CF53
:1007100000F0E4CFD9FF1200620ED36EFF0E926E8E
:100720000F0E936EFF0E946E816AF4EC0AF05AEC91
:1007300009F0E5EC0AF02EEC0BF036EC0BF0816AD8
:10074000F26AF28C9D84F18CF288F28E090EE56ECD
:100750008FEC09F0006EF3CF01F0E12A000E036E7A
:10076000800E026E800E046E0150E56E0050E56E44
:10077000000EE56E0450E56E0350E56E0250E56E26
:1007800015EC00F0060EE1260001866B000E036EEC
:10079000800E026E800E046EE56E0350E56E025010
:1007A000E56E000EE56E000EE56E99EC04F0050EA8
:1007B000E1260050200F026E000E0120036E02346D
:1007C000016E0334006E013600360134030B016EF6
:1007D000000E036E800E026E800E046E0150E56EF8
:1007E0000050E56E000EE56E0450E56E0350E56EB8
:1007F0000250E56E15EC00F0060EE1260001866B56
:10080000000E036E800E026E800E046EE56E0350C5
:10081000E56E0250E56E010EE56E000EE56E99EC98
:1008200004F0050EE1260038F00B816E8FD7120020
:10083000D9CFE5FFE1CFD9FF00C0E5FF01C0E5FF5B
:1008400002C0E5FF03C0E5FF04C0E5FF05C0E5FF0A
:1008500006C0E5FF07C0E5FF020EDBCF00F0030E88
:10086000DBCF01F0040EDBCF02F0050EDBCF03F08F
:10087000060EDBCF04F0070EDBCF05F0080EDBCF52
:1008800006F0090EDBCF07F01AEC0AF003A003D044
:10089000020EC86E02D0090EC86E56EC0BF0005066
:1008A000E56E03EC0BF0E12A03A208D00250006EC3
:1008B000036A0050E56E03EC0BF0E12A0150E56E8F
:1008C00003EC0BF0E12A04C000F005C001F006C003
:1008D00002F007C003F003C004F00306045013E065
:1008E00000C0E9FF01C0F3FF0250C4EC0AF0046E3F
:1008F000002AD8B0012AD8B0022A0450E56E03ECD1
:100900000BF0E12AE8D74AEC0BF0E86AE4CF07F0F5
:10091000E4CF06F0E4CF05F0E4CF04F0E4CF03F039
:10092000E4CF02F0E4CF01F0E4CF00F0E4CFD9FF50
:100930001200D9CFE5FFE1CFD9FF00C0E5FF01C02C
:10094000E5FF02C0E5FF03C0E5FF04C0E5FF020EBE
:10095000DBCF00F0030EDBCF01F0040EDBCF02F0A3
:10096000050EDBCF03F0060EDBCF04F01AEC0AF025
:10097000090EC86E56EC0BF0C60EE56E03EC0BF0DC
:10098000E12A000EE56E03EC0BF0E12AFE0EE56EA7
:1009900003EC0BF0E12A0150400DF3CF01F0800E83
:1009A0000126015000260050E56E03EC0BF0E12A11
:1009B00002C000F003C001F004C002F000C0E9FF73
:1009C00001C0F3FF0250C4EC0AF0036E03500BE0C9
:1009D000002AD8B0012AD8B0022A0350E56E03ECF1
:1009E0000BF0E12AEBD7FF0EE56E03EC0BF0E12AEA
:1009F0004AEC0BF0000EE56E0A0EE56EC2EC09F053
:100A0000020EE126E4CF04F0E4CF03F0E4CF02F0DD
:100A1000E4CF01F0E4CF00F0E4CFD9FF1200D9CF4A
:100A2000E5FFE1CFD9FF00C0E5FF01C0E5FF02C04F
:100A3000E5FF03C0E5FF04C0E5FF05C0E5FF06C014
:100A4000E5FF07C0E5FF08C0E5FF09C0E5FF0AC0F4
:100A5000E5FF0BC0E5FF020EDBCF00F00050E56EB6
:100A6000CFEC07F0016EF3CF02F0E12A036A046ACB
:100A7000002A002A0050E56ECFEC07F0006EF3CF9D
:100A800005F0E12A066A076A05500B6E00500A6EEF
:100A9000086A096A08500112095002120A5003122A
:100AA0000B50041204C0E9FF03C0F4FF02C0F3FFBF
:100AB0000150E4CF0BF0E4CF0AF0E4CF09F0E4CF2B
:100AC00008F0E4CF07F0E4CF06F0E4CF05F0E4CF80
:100AD00004F0E4CF03F0E4CF02F0E4CF01F0E4CF80
:100AE00000F0E4CFD9FF1200D9CFE5FFE1CFD9FF65
:100AF00000C0E5FF01C0E5FF02C0E5FF03C0E5FF60
:100B000004C0E5FF05C0E5FF06C0E5FF020EDBCF30
:100B100000F0030EDBCF01F0040EDBCF02F0050E78
:100B2000DBCF03F0046A056A0344010B066E06B0CE
:100B300011D00250022603360350015C02E102503C
:100B4000005C04E2D8900332023204D0052A05C0CA
:100B500004F0EAD70350015C02E10250005C04E3B8
:100B60000250005E0350015AD8900332023204C092
:100B700005F004060550EEE101C0F3FF0050E4CF9C
:100B800006F0E4CF05F0E4CF04F0E4CF03F0E4CFC7
:100B900002F0E4CF01F0E4CF00F0E4CFD9FF12007F
:100BA000D9CFE5FFE1CFD9FF00C0E5FF01C0E5FFE8
:100BB00002C0E5FF03C0E5FF04C0E5FF05C0E5FF97
:100BC00006C0E5FF07C0E5FF020EDBCF00F0030E15
:100BD000DBCF01F0040EDBCF02F0050EDBCF03F01C
:100BE000046A056A100E066E0144010B076E010EC1
:100BF000071600500026013604500426053607501B
:100C0000D8A404800350055C02E10250045C05E3B3
:100C10000250045E0350055A0080062EE5D701C03D
:100C2000F3FF0050E4CF07F0E4CF06F0E4CF05F087
:100C3000E4CF04F0E4CF03F0E4CF02F0E4CF01F01E
:100C4000E4CF00F0E4CFD9FF1200D9CFE5FFE1CF28
:100C5000D9FF00C0E5FF01C0E5FF02C0E5FF020EBD
:100C6000DBCF00F000380F0B016E300E01263A0E7C
:100C7000015C02E3070E012601500001936F0F0E85
:100C80000014016E300E01263A0E015C02E3070EDD
:100C9000012601500001946F9569000E016E930EBC
:100CA000006E800E026E030EE56E0250E56E01507E
:100CB000E56E0050E56E000EE56E000EE56E000E6E
:100CC000E56EC60EE56E18EC04F0080EE126000E87
:100CD000E56E0A0EE56EC2EC09F0020EE126E4CFE5
:100CE00002F0E4CF01F0E4CF00F0E4CFD9FF12002E
:100CF000D9CFE5FFE1CFD9FF00C0E5FF01C0E5FF97
:100D000002C0E5FF03C0E5FF04C0E5FF05C0E5FF45
:100D100006C0E5FF020EDBCF00F0030EDBCF01F0D3
:100D2000040EDBCF02F0050EDBCF03F0060EDBCFA7
:100D300004F00150056E0250066EE56E0550E56E3A
:100D40000050E56E94EC07F0030EE126002A002A1D
:100D50000350016E0450026E036A046A0250E56E8D
:100D60000150E56E0050E56E94EC07F0030EE126AD
:100D7000E4CF06F0E4CF05F0E4CF04F0E4CF03F0D5
:100D8000E4CF02F0E4CF01F0E4CF00F0E4CFD9FFEC
:100D900012007A0EF66E160EF76E000EF86E09004F
:100DA000F550056E0900F550066E055002E106503B
:100DB0003BE00900F550006E0900F550016E090096
:100DC000F550026E09000900F550E96E0900F55072
:100DD000EA6E090009000900F550036E0900F5509C
:100DE000046E09000900F6CF07F0F7CF08F0F8CF3E
:100DF00009F000C0F6FF01C0F7FF02C0F8FF035082
:100E000002E1045007E00900F550EE6E0306F8E237
:100E10000406F9D707C0F6FF08C0F7FF09C0F8FFBE
:100E20000506C4E20606C5D71200D9CFE5FFE1CF1B
:100E3000D9FF00C0E5FF01C0E5FF02C0E5FF03C028
:100E4000E5FF04C0E5FF05C0E5FF020EDBCF00F0C3
:100E5000030EDBCF01F0040EDBCF02F0050EDBCF7B
:100E600003F0046A0350045C14E200C0E9FF01C00F
:100E7000F3FF0250C4EC0AF0056E002AD8B0012A34
:100E8000D8B0022A0550E56EB2EC0AF0E12A042A35
:100E9000E9D7E4CF05F0E4CF04F0E4CF03F0E4CFEA
:100EA00002F0E4CF01F0E4CF00F0E4CFD9FF12006C
:100EB000D9CFE5FFE1CFD9FF00C0E5FF01C0E5FFD5
:100EC00002C0E5FF020EDBCF00F000500001966F7C
:100ED0009769000E016E960E006E800E026E020E75
:100EE000E56E0250E56E0150E56E0050E56E000EB5
:100EF000E56E000EE56E000EE56EC60EE56E18ECB2
:100F000004F0080EE126000EE56E0A0EE56EC2EC56
:100F100009F0020EE126E4CF02F0E4CF01F0E4CFC5
:100F200000F0E4CFD9FF1200D9CFE5FFE1CFD9FF20
:100F300000C0E5FF01C0E5FF02C0E5FF020EDBCF08
:100F400000F0030EDBCF01F0040EDBCF02F0A69E13
:100F5000A69CA684F29E00C0A9FF0150A86E550E63
:100F6000A76EAA0EA76EA682A6B2FED70028A96E0B
:100F70000250016E026A0150A86E550EA76EAA0EAD
:100F8000A76EA682A6B2FED7A694F28EE4CF02F098
:100F9000E4CF01F0E4CF00F0E4CFD9FF1200D9CFC5
:100FA000E5FFE1CFD9FF00C0E5FF01C0E5FF02C0CA
:100FB000E5FF03C0E5FF04C0E5FF05C0E5FF020E45
:100FC000DBCF00F0A69CA69E00C0A9FFA680A8CFFC
:100FD00001F0026A0028A96EA680A8CF00F0036A7B
:100FE0000050056E046A045001120550021202C03E
:100FF000F3FF0150E4CF05F0E4CF04F0E4CF03F0B9
:10100000E4CF02F0E4CF01F0E4CF00F0E4CFD9FF69
:101010001200D9CFE5FFE1CFD9FF00C0E5FF01C045
:10102000E5FF02C0E5FF03C0E5FF020EDBCF00F0E5
:10103000030EDBCF01F0040EDBCF02F000C0E9FFAE
:1010400001C0F3FF0250C4EC0AF0036E035010E03D
:10105000ACA2FED700C0E9FF01C0F3FF0250C4EC10
:101060000AF0AD6E002AD8B0012AD8B0022AE6D71D
:10107000E4CF03F0E4CF02F0E4CF01F0E4CF00F0DE
:10108000E4CFD9FF1200D9CFE5FFE1CFD9FF00C0EF
:10109000E5FF01C0E5FF02C0E5FF03C0E5FF020E6A
:1010A000DBCF00F0030EDBCF01F0026A036A01BE62
:1010B0000CD0D89001360150005C03E2D890013288
:1010C00004D0032A03C002F0F2D70150005C02E30F
:1010D0000150005ED890013202C003F002060350B6
:1010E000F4E10050E4CF03F0E4CF02F0E4CF01F0EC
:1010F000E4CF00F0E4CFD9FF120000C0E5FF01C04B
:10110000E5FF02C0E5FF03C0E5FF24EC09F0006E37
:10111000F3CF01F0F4CF02F0E9CF03F0000EE56E5B
:101120000F0EE56E420EE56E400EE56E0350E56E65
:101130000250E56E0150E56E0050E56EFFEC02F0E6
:10114000006EF3CF01F0F4CF02F0E9CF03F0080E08
:10115000E12601C0F3FF0050E4CF03F0E4CF02F03A
:10116000E4CF01F0E4CF00F0120000C0E5FF01C0C1
:10117000E5FF02C0E5FF03C0E5FF24EC09F0006EC7
:10118000F3CF01F0F4CF02F0E9CF03F0000EE56EEB
:10119000000EE56E030EE56EE80EE56E0350E56E9B
:1011A0000250E56E0150E56E0050E56EFFEC02F076
:1011B000006EF3CF01F0F4CF02F0E9CF03F0080E98
:1011C000E12601C0F3FF0050E4CF03F0E4CF02F0CA
:1011D000E4CF01F0E4CF00F01200D9CFE5FFE1CF7A
:1011E000D9FF00C0E5FF01C0E5FF02C0E5FF03C075
:1011F000E5FF04C0E5FF020EDBCF00F0030EDBCFFE
:1012000001F0026A080E036E800E0014046ED8907E
:101210000036D89002360450D8A402800150025CF7
:1012200003E30150025E0080032EEED70050E4CFAE
:1012300004F0E4CF03F0E4CF02F0E4CF01F0E4CF18
:1012400000F0E4CFD9FF120000C0E5FF01C0E5FFC8
:1012500002C0E5FF03C0E5FF04C0E5FF05C0E5FFF0
:10126000B2CF00F0B3CF01F098C002F099C003F004
:10127000B2CF04F0B3CF05F00150055C02E100509D
:10128000045C04E298C002F099C003F003C0E9FFD7
:1012900002C0F4FF05C0F3FF0450E4CF05F0E4CF33
:1012A00004F0E4CF03F0E4CF02F0E4CF01F0E4CFA8
:1012B00000F0120000C0E5FF01C0E5FF02C0E5FF3D
:1012C000FE0E0001906F010E916F9269000E016E8B
:1012D000900E006E800E026E030EE56E0250E56EFB
:1012E0000150E56E0050E56E000EE56E000EE56EF5
:1012F000000EE56EC60EE56E18EC04F0080EE12651
:10130000000EE56E0A0EE56EC2EC09F0020EE12653
:10131000E4CF02F0E4CF01F0E4CF00F01200D9CF27
:10132000E5FFE1CFD9FF00C0E5FF01C0E5FF02C046
:10133000E5FF03C0E5FF020EDBCF00F00044E84408
:10134000FC0B016E030E0110C26EC2B2FED7C4CFF9
:1013500000F0016A0050036E026AC3CF00F0016A18
:10136000005002260150032203C0F3FF0250E4CFD5
:1013700003F0E4CF02F0E4CF01F0E4CF00F0E4CFDB
:10138000D9FF1200D9CFE5FFE1CFD9FF00C0E5FFBB
:1013900001C0E5FF02C0E5FF03C0E5FF020EDBCFA1
:1013A00000F0030EDBCF01F000C002F001C003F03B
:1013B000FF0E0026D8A001060250031006E0FA0E28
:1013C000026E0000022EFDD7EFD7E4CF03F0E4CF8A
:1013D00002F0E4CF01F0E4CF00F0E4CFD9FF120037
:1013E000E8CFE5FFD8CFE5FFE0CFE5FFF3CFE5FF9E
:1013F000F4CFE5FFE9CFE5FFEACFE5FFFACFE5FF60
:10140000FBCFE5FF9EA403D05CEC0BF09E94E4CFF1
:10141000FBFFE4CFFAFFE4CFEAFFE4CFE9FFE4CF3C
:10142000F4FFE4CFF3FFE4CFE0FFE4CFD8FFE4CF55
:10143000E8FF100000C0E5FF01C0E5FF02C0E5FFC6
:10144000FF0E006E1F0EC514016E026AC7B4022A99
:1014500002500112015003E000060050F3E100C009
:1014600001F00050D8B4D5EC0AF00150D880E866FD
:10147000D890016A01360150E4CF02F0E4CF01F0C8
:10148000E4CF00F01200D9CFE5FFE1CFD9FF00C0D3
:10149000E5FF01C0E5FF020EDBCF00F0030EDBCF5E
:1014A00001F0A69EA69CA684F29E01C0A8FF00C0E3
:1014B000A9FF550EA76EAA0EA76EA682A6B2FED7EA
:1014C000A694F28EE4CF01F0E4CF00F0E4CFD9FF90
:1014D0001200D9CFE5FFE1CFD9FF00C0E5FF01C081
:1014E000E5FF020EDBCF00F01AEC0AF0C5861AEC1D
:1014F0000AF0C9CF01F01AEC0AF0005002E0C59AD8
:1015000001D0C58AC5880150E4CF01F0E4CF00F0D6
:10151000E4CFD9FF1200D9CFE5FFE1CFD9FF00C05A
:10152000E5FF020EDBCF00F0A69CA69E00C0A9FF3F
:10153000A680A850E4CF00F0E4CFD9FF120000C08D
:10154000E5FF01C0E5FF1F0EC514006E016AC7B4B8
:10155000012A015000120050F6E1E4CF01F0E4CF7F
:1015600000F01200D9CFE5FFE1CFD9FF00C0E5FFC1
:10157000020EDBCF00F0ACA2FED700C0ADFFE4CF7F
:1015800000F0E4CFD9FF1200E8AE04D0F3CFEAFFB9
:10159000EE501200E8BC08D0E9CFF6FFF3CFF7FF1A
:1015A000F86E0900F55012001200818AC69A9496CE
:1015B000828682B803D082968286FBD794988298DE
:1015C000828894869488C68A1200200EAC6E900E93
:1015D000AB6E0C0EAF6E000EE56E010EE56EC2EC4A
:1015E00009F0020EE12612003F0EC716280EC66E45
:1015F000C56A090EC86E948694889E96A196D5EC0D
:101600000AF0819A1200D9CFE5FFE1CFD9FF020E8F
:10161000DBCFC9FF1AEC0AF0E4CFD9FF120012EEBB
:10162000FFF022EEFFF0F86AA68EA69CC9EC06F049
:101630008CEC03F0FFD7E8AE05D0F3CFEAFFE4CFA0
:10164000EEFF1200E8AC1200120000C0E5FF006AD5
:101650009EBA002A0050E4CF00F01200810EB16E55
:10166000B36AB26A0001986B996B1200010EC26EE8
:10167000050EC16E940EC06E12000100CA16000065
:101680009A00000001000000B36AB26A0001986B82
:10169000996B12001AEC0AF0C584C5B4FED712008B
:1016A0001AEC0AF0C582C5B2FED712001AEC0AF095
:1016B000C580C5B0FED712000001982B01E3992B1D
:0C16C00012009EAAFED7AE5012000000DF
:00000001FF
